:100000000CC024C023C022C021C020C01FC01EC0FD
:100010001DC01CC08198A6AFB80011241FBECFE937
:10002000CDBF10E0A0E6B0E0E0E0F2E002C0059055
:100030000D92AA36B107D9F710E0AAE6B0E001C0E8
:100040001D92AB36B107E1F724D0D8C0D9CF2AE74B
:1000500033E003C0F9013197F1F70197D8F708951C
:1000600080916A008F5F80936A0080916A00893076
:1000700010F010926A00089581E687B9A29A86EC82
:1000800086B9089537980895369A3699FECF85B186
:10009000089582E087BB83E28FBD81E083BFECDF00
:1000A000479A85B7877E85BF80916C00882329F0A9
:1000B00010926B0010926A0009C080916B008093CF
:1000C0006A00CEDF80916A0080936B0010926C0012
:1000D000E0916A00F0E0E05AFF4F808189BD10E0B6
:1000E00088E7F82E0FEFCCE2D1E080916A008430EF
:1000F00040F485B7806285BF889585B78F7D85BFC1
:1001000051C080916A00853080F409BD8AE090E09A
:100110009EDF19BC80EF90E09ADF09BD8AE090E095
:1001200096DF19BC84EE92E03CC080916A00883072
:1001300098F409BD8AE090E08ADF19BCE0916A007A
:10014000F0E0E05AFF4F808190E0009709F029C06D
:10015000CE010197F1F726C080916A00893010F531
:1001600019BC88EE93E073DF8FDF8EDFE4E1F0E00F
:10017000E12C9491981708F4E394319690E0E931DA
:10018000F907B9F7D12C09C0F9BC84E690E05FDF2C
:1001900019BC80E991E05BDFD394DE10F5CF88EEE7
:1001A00093E055DF349BA1CF6FDF90E020916A0090
:1001B000211103C021E730E002C02BE730E08217B5
:1001C0009307CCF41F5F1330B8F080916A00882346
:1001D00019F010926A000CC019BC85B7877E806147
:1001E00085BF85B7806285BF889585B78F7D85BFC0
:1001F00088EE93E02CDF10E0369A77CFF894FFCFAB
:0A020000061E78FFFFF05A1F780079
:00000001FF
